:030000000219FDE5
:03000B000200AA46
:03002B0002018A45
:03005B0002034459
:0300730002033154
:1000800002030406080C10182030406080040608A3
:100090000C10182030406080A0C00003070F1F0D17
:1000A0000D04050D050305030302C2AF306308C24A
:1000B0006385798AD2AF32C0D0C0E0206221E525C5
:1000C0006016E473E525F4C3334009758A00D263F2
:1000D000F57901D6F58AD262D0E0D0D0D2AF32C362
:1000E000E526334009758A00D263F57901F0F58A77
:1000F000C262E526F4603030682620720DD0E0D070
:10010000D0C295C294C293D2AF32C295C294C29368
:10011000206F0D20650A7414D5E0FDE57BF4529044
:10012000D0E0D0D0D2AF32758A00D263757900C2E8
:100130008DD262212001C4306805206502D295016C
:10014000C4306805206502D29401C430680520657A
:1001500002D29301C4D29230680A2065077410D588
:10016000E0FDD29501C4D29130680A206507741071
:10017000D5E0FDD29401C4D290D29230680A2065B5
:10018000077410D5E0FDD29301C4C2AFC2AD53E6EF
:10019000EFC0D0C0E0D2D3D2AFE57A6009E5776096
:1001A0000575770041DE757701C2CEE52A6007202C
:1001B000744F152A41017800790020742EE58030B3
:1001C0007E01F430E70278FF53DACF207E0343DA72
:1001D00020307E0343DA10C2D8C271E580307E0140
:1001E000F430E70279FFC3E89970CB306103752AD8
:1001F00018207403752A18885CD270E86003755F54
:100200000020740DE52B6004152B411143DA01C267
:10021000D82070024180A85C206102C27020743630
:100220007982B70431C3E894F0400374F0F8E8C46D
:10023000540F28F87984B703024156C313C31387B8
:1002400021200802C313200A06C3C898F841562883
:10025000F8500374FFF88822E52D54066022206BC5
:100260001FE536C333C333F8E564C313C313F9C3BF
:10027000952240028922E82522F52250037522FFAB
:100280007882B60459852224A824C3E524956140C8
:1002900002A861C3E895634002A8638825E56670FB
:1002A0000241D1C3E8AA669A5003E8FAE4F9EAC326
:1002B00033FBE568F45B29400D2567F8E5676002CC
:1002C0001567400B41D10AC3E5679A50020567786C
:1002D000FF8826C26FC3E52694F84002D26F20CF74
:1002E0000AD0E0D0D043E610D2AD32C2CF053AE515
:1002F0007A6009E57860057578006127757801787E
:1003000001E52A6005307402152AC3E55C940140BA
:1003100005755F006127756000756900E55F240160
:10032000F55F5003755FFFD0E0D0D043E610D2AD4B
:1003300032C2AF53E67F7592FA7593FFC260759132
:1003400004D2AF32C2AF53E6EFC2ADC0D0C0E0C0FE
:10035000F0D2D3D2AFA8FBA9FCE57A6007C3E913BA
:10036000F9E813F8C2D830710261B653DACF207EB3
:100370000343DA10307E0343DA20D271E580307E09
:1003800001F420E702618D88278928A1E353DACFA1
:10039000207E0343DA20307E0343DA10C2D8C271D4
:1003A000307402A1CF7800E580307E01F430E7029E
:1003B000A1CF885CA1B753DACF207E0343DA203087
:1003C0007E0343DA10C271206102818F53DACF209D
:1003D0007E0343DA10307E0343DA20C2D8D271881C
:1003E000578958C3E89555F8E99556F97B007E087A
:1003F0007A00C3E8948CE994005005755B00818114
:10040000882178A2E6A8216055C3E894C8E9940041
:100410005008E4D2E4FB7A0A815CC3E89468E9946A
:10042000015008E4D2E3FB7A0F815CC3E894D0E981
:1004300094025008E4D2E2FB7A1E815CC3E894A0E7
:10044000E994055008E4D2E1FB7A3C815CC3E8946E
:1004500098E994085008E4D2E0FB7A787E00C3E87B
:100460009559FCE9955AFD30E70AECF42401FCEDBE
:0E047000F43400FD755B00C3EC9AED9E500362
:10047E00755B018859895A8557558558567802A15A
:10048E00B7C3E89527F8E99528F9307C02A19B308F
:10049E007B02A19B307A02A19420750281B2E9FD04
:1004AE00E8FC81D1E9C313F9E813F8307902A1947D
:1004BE00E9C313F9E813F8307802A194E9C313FDE8
:1004CE00E813FC20612CC3EC941CED9402400281D5
:1004DE00E8ED701EC3EC94C850180529E52970028A
:1004EE001529C3E529940A5002A1CF755C00D2707C
:1004FE00A1CFE529600215297888E6F97400207FDE
:10050E00087896B90302789EE624FAFEE43400FFDA
:10051E00C3EC9EFCED9FFD9208B90310A208500794
:10052E00207609D276A13A307602C276A20850160B
:10053E00B9030DECF42401FCEDF43400FD02055476
:10054E0078007900A19BB90315EC33FCED33FDC3A4
:10055E00EC940AFCED9400FD50047C007D00C3EC8D
:10056E0094FFED9400400678FF7900A19BEC857214
:10057E00F0A4C5F0A2F733F8790040030205B7786E
:10058E00FF79000205B7E9C313F9E813F8307C0EC2
:10059E00E9600278FFC3E81338F8E43400F9C3E8E1
:1005AE0094FFE99400400278FF885CD270206102CB
:1005BE00A1CF741FF4552F4BF52FC274EB7002D2DE
:1005CE0074752A18307403752A0A306102A1E3206B
:1005DE00740353DAFE207403752B06D0F0D0E0D0EE
:1005EE00D0D2AD43E610327901020613790302062A
:1005FE0013790A020613791E020613796402061392
:10060E0079C80206137817E4D5E0FDD8FAD9F62298
:10061E007A147B7802063A7A107B8C02063A7A0DAF
:10062E007BB402063A7A0B7BC802063AE573D5E034
:10063E0001227902E4D291D5E0FDD294D5E0FDC23B
:10064E0094D5E0FDC291D5E0FDE920E002D29530CF
:10065E00E002D293E573D5E0FDE920E002C29530C9
:10066E00E002C2937496D5E0FDD9C9EAF8D5E0FD53
:10067E00D8FBDBB8D29122C37C007D0075F000055B
:10068E00F0EA33FAEB33FB50F6EB13FBEA13FAC343
:10069E00E9FFE8FEE89AF8E99BF95004EFF9EEF865
:1006AE00B3EC33FCED33FDD5F0DFEDF9ECF822E8D9
:1006BE0089F08A20D2D4F8A9F07B0030F70B7BFFAB
:1006CE00F42401F8E9F43400F9E88520F0A4ADF043
:1006DE00F8E98520F0A4AFF0FEED2EF974003FFA94
:1006EE007C04C3EA13FAE913F9E813F8DCF48BF08F
:1006FE0030F70AE8F42401F8E9F43400F9E889F057
:10070E00C2D4F8A9F0227882B6040302076FC3E5BB
:10071E005C94014003020739852224E4F544F54533
:10072E00F546F547F548C26E02076F7882E6FCD2B1
:10073E006EE522F523783879C7AA40AB41C3EB1397
:10074E00FBEA13FAEC146013C3EB13FBEA13FAEC97
:10075E0014146007C3EB13FBEA13FAD1858844899E
:10076E004522C3E5449523F8E5459400F9500CC3A2
:10077E00E89480E994FF40160207A0C3E8947FE94D
:10078E00940050030207A0787F79000207A07880BA
:10079E0079FF8849894A22E5492546F8E54A3547D1
:1007AE00F9854A20E4300701F43548FA30E709C3E9
:1007BE00EA94F040150207DEC3EA940F50030207D5
:1007CE00DE78FF79FF7A0F0207DE780079007AF083
:1007DE00C3E5249561500AC374019524500B02079A
:1007EE00FCE54A20E70E0207FCE54A30E70688469C
:1007FE0089478A482278A5E6FAC3E54933F8E54ADF
:10080E0033F91206BDE930E70BC3E89480E994FF93
:10081E0040130137C3E8947FE99400500201377802
:10082E007F79000137788079FFE820E715C3E5234B
:10083E0098F84009C3E89401400302085E7801026B
:10084E00085EE8F424012523F8400302085E78FFD1
:10085E00884B2278A6E6FAA847A9481206BDE930C9
:0F086E00E70CC3E89401E994FF4016020893C316
:10087D00E894FFE99400500302089378FF79000291
:10088D000893780179FFE920E715C3E54B98F84007
:10089D0009C3E8940140030208BA78010208BAE8D6
:1008AD00F42401254BF840030208BA78FF8824226E
:1008BD0078FF20692879A1E76023E541601F74FF67
:1008CD008541F0848539F0306A0375F005A4F8C5CB
:1008DD00F0600278FFC3E895645002A86488632233
:1008ED00C3E54094C8E5419400E56350031401FE4F
:1008FD00046002F563220209062275E890227883CE
:10090D00E6FF30EDF9A8BDA9BE0570C3E5709408EA
:10091D004052757000E9FA79A0E76044EA7007E586
:10092D0071601B02093FC3E895716010E5715006B7
:10093D00600C1402094B0460F902094BE571F57165
:10094D00C39472401B7561C0C394044013756180DC
:10095D00C39404400B756140C3940440037561005A
:10096D0075BB0622E5612410500274FFF561798292
:10097D00B704022198C3A861E524985002A824C3A6
:10098D00E895634002A86388258826E570B40703BF
:10099D0075BB1022743279A787F0A4C5F0A2F73386
:1009AD00F8C3E895614002A86188228824882588CB
:1009BD00268864227540007541F022C2AF75C820AB
:1009CD00A8CCA9CDAA3A30CF010A75C824D2AFC39D
:1009DD00EA13FAE913F9E813F8AB3BAC3C883B8911
:1009ED003CC3E89BF8E99C20690A547FF930660204
:1009FD0041E74141AD3D8A3DF9EA9D547FFA6006DC
:100A0D0078FF79FF4126AE3EAF3F8B3E8C3FA83B32
:100A1D00A93CC3E89EF8E99FF9C3E54113FBE54006
:100A2D0013FAE82AF540E93BF54150067540FF758C
:100A3D0041FF418EAA40AB41AC40AD417E047F02E7
:100A4D00C3EB9404400D1E1FC3EB94084005206AB0
:100A5D00021E1FC3ED13FDEC13FCDEF7C3EA9CFA77
:100A6D00EB9DFBEF6009C3E913F9E813F8DFF7EA33
:100A7D0028FAEB39FB8A408B4150067BFF8B408B6C
:100A8D0041C3EB94025002D2663069047F0341B931
:100A9D007892E6FFC3E537948240110FC3E5379492
:100AAD00A040010FC3EF940640027F057E02E54191
:100ABD00C4540FF9E541C454F0F8E540C4540F286F
:100ACD00F8C3E89EFAE99400FB4009C3EA9402EBEF
:100ADD00940050047A02E4FB6133AA40AB41EBC4AD
:100AED00FEEAC4540F4EFCC3EA9CFAEB9400FBC320
:100AFD00E813C313F8EA28FAEB3400FB8A408B4164
:100B0D00C3EB94024002C2667802EBC4FE7B00EA9E
:100B1D00C4540F4EFAC3EA98FA4005C3940250022A
:100B2D007A027892E6FF30600261338551928552E8
:100B3D0093D26043E680C3E49AF8E49BF9C3E833AB
:100B4D00F8E933F930660261C6E8FAE9FBD3E91337
:100B5D00FDE813FC88518952C3EF94036038EF20F0
:100B6D00E00DE82CF8E93DF9ECFAEDFB020B8FE80E
:100B7D0028F8E939F9C3E82402F8E93400F97AFED6
:100B8D007BFFC3EF9403400E8A538B54884D894EDF
:100B9D008C4F8D5061FA885389548A4D8B4E8C4FF2
:100BAD008D503069127553F07554FF754FF07550B7
:100BBD00FF7551F07552FF61FAE8FAD3E813FC881E
:100BCD0051C3EF94036020EF20E007E82CF8ECFA16
:100BDD0061E6E8282402F87AFEC3EF940340088A00
:100BED0053884D8C4F61FA88538A4D8C4FE568C3FD
:100BFD00335002646BF5683060028104753402D2A3
:100C0D006043E680E52D5406602DA840A941C3E957
:100C1D0013F9E813F8306904E92440F9C2AF53E63B
:100C2D007F759100C3E498F594E499F59575910459
:100C3D00D26043E680D2AF22D264754300752000A6
:100C4D00306C03752040020C64D26475430075202E
:100C5D0040306C0375200078017901206620E52D68
:0F0C6D0054066002C2647914E541C31370010498
:100C7C00F8C3941440027814306904781B791BC3B0
:100C8C00E833F8C3E933F9206010E543600C3069B0
:100C9C0003D53404D26DA11A910C0543E59B544045
:100CAC00B52002A10430690908C3E89940011881F4
:100CBC009320640A08C3E899400281648193C2645A
:100CCC00C2AF53E67F75910030661275940075952E
:100CDC00F0759104D26043E680D2AF8164E5417E29
:100CEC00FFC3334009C3334005C3334001FEC3E4A3
:100CFC009E759400F59581DDC3E533940150028116
:100D0C00643064028164D802A1188193C26DC2AFB1
:100D1C0053E67F75910085539485549575910485A0
:100D2C004D92854E93D26043E680D2AFE52D5406AA
:100D3C006008206A020533020D56306D0D206C0AD6
:100D4C002064071581158102162522780030640273
:100D5C007801E53775F007A4F9E5F028F5F0E9A27C
:100D6C00F013A2F113A2F213F537C3947850037564
:100D7C003778C3E53795384008D265C295C294C21E
:100D8C0093306002A18D854F92855093D26043E6DB
:100D9C008022207D16C2AF754202D291C29230627F
:100DAC0002D293D2AF759F11020F96C2AF75420259
:100DBC00D291C290306202D295D2AF759F11020FC0
:100DCC0096307245207D22C2AF7542039001667544
:100DDC007B02C293D290D292306204D294A1EDC223
:100DEC0091D2AF759F01020F96C2AF75420390016D
:100DFC0066757B02C295D292306204D294C10DC248
:100E0C0091D2AF759F21020F96207D17C2AF75420C
:100E1C0003900141C293306202D294D2AF759F010C
:100E2C00020F96C2AF754203900141C29530620227
:100E3C00D294D2AF759F21020F96207D16C2AF754A
:100E4C004204D292C290306202D294D2AF759F21EA
:100E5C00020F96C2AF754204D290D292C292306207
:100E6C0002D294D2AF759F01020F96307243207D4F
:100E7C0020C2AF754205900155757B04C294D29186
:100E8C00306204D295C195C292D2AF759F11020FF8
:100E9C0096C2AF754205900177757B01C294D291D1
:100EAC00306204D293C1B5C290D2AF759F11020FBC
:100EBC0096207D17C2AF754205900137C2943062FF
:100ECC0002D295D2AF759F11020F96C2AF75420533
:100EDC0090014BC2943062EBD293D2AF759F11024A
:100EEC000F96207D18C2AF754206D290D292C29155
:100EFC00306202D295D2AF759F01020F96C2AF75C8
:100F0C004206D292C291306202D293D2AF759F2127
:100F1C00020F96307246207D20C2AF7542019001BF
:100F2C0077757B01C295D292306204D293E13DC2B7
:100F3C0090D2AF759F21020F96C2AF7542019001FE
:100F4C0055757B04C293D290D292306205D2950231
:100F5C000F60C292D2AF759F01020F96207D17C20F
:100F6C00AF75420190014BC295306202D293D2AF61
:100F7C00759F21020F96C2AF754201900137C29343
:100F8C00306202D295D2AF759F01C26522900135B5
:100F9C00757B00C295C294C293D292D291D290C268
:100FAC006222788076090876090876040876FF08AC
:100FBC0076030876FF08760A087603087601087629
:100FCC0001788C76010876FF0876FF0876FF0876A4
:100FDC00FF0876FF0876030876FF0876FF0876FF91
:100FEC000876250876D00876280876500876040806
:100FFC0076FF08760208760008767A0876FF08767F
:10100C0001087601087600087603087600227887B6
:10101C00E6FFC272BF0302D2727888E6C394036003
:10102C0008C27DE630E102D27DC27E7889E630E1ED
:10103C0002D27EC3EF94026008758E01D273021047
:10104C0052758E00C273227880E6149000809378DB
:10105C00A5F67881E6149000809378A6F67886E65B
:0E106C001490008D9378A7F67886E6F539C3C8
:10107A0094025003753902789CE67538FFB402036E
:10108A007538A0B4030375388278A3E61490009AE1
:10109A0093F566120F9922227896E6FA7897E6FB7C
:1010AA007888E6B40305C3EB940EFB307F047A001C
:1010BA007BFFC3EB9AFCC3948250027C8275720058
:1010CA000572EC8572F0A4C3E5F0947D40F222D259
:1010DA007F11A21206041206047A007B007C101209
:1010EA0005FAE55C2AFA74003BFBDCF37C04C3EBEB
:1010FA0013FBEA13FADCF7FEC27F11A222757C0009
:10110A00757D00E5EF20E6037520000520903FFF7E
:10111A00E520146006901FFF1460009304600375B5
:10112A00EF1653D9BF7581C043FF801205F575EFDD
:10113A000643B203E5B3240220E70DF521E5E320D7
:10114A00E0068521B343E301120F997580FF75A468
:10115A000075F19075D47F75908775A5BF75F2BF3C
:10116A0075D50075A60175E241120F99E4F8F6D813
:10117A00FD756801120FAE12167E78988673753067
:10118A0001C2AF12060E12061E120604120625121C
:10119A00060412062C120604C2AF757C00757D0087
:1011AA0078FA79FA308707D9FBD8F7021C00111AA6
:1011BA00115311A111A278988673120F9975A9007B
:1011CA0075B680757A0075881075890275C8247598
:1011DA00910475D84075A82275B80275E690759B7A
:1011EA0080759D0075D10E75BC5875BB0675BA1110
:1011FA0075E8801205F5D2AF12090375360053DA85
:10120A00CF207E0343DA20307E0343DA1043DA012B
:10121A00C2D8C27112060ED2617B037A0CE55B70EA
:10122A00077A0CDB030211A21206042070030211D2
:10123A00A2C270E55CC3940240E1E52F541F855EAB
:10124A005DF55EB55DD5DAD5C26153DACF207E038E
:10125A0043DA20307E0343DA10C2D8C27178A2E69C
:10126A007008D274E52F54E0F52FC2757529001263
:10127A000609307409C3E529940A4002D275120599
:10128A00FA78023074027800C3E55C9840F0C2AF85
:10129A0012061E12061E12061ED2AF12060E754C3A
:1012AA00007888E6B40302619E1205FA788CE6C3D8
:1012BA009401500302139EE530C3940150030213B4
:1012CA009E757CA5757DF1207435C3E55C94FF504D
:1012DA000302139EC2AF120633D2AF120609C3E548
:1012EA005C940150EFC2AF12061E1205FF12061ED1
:1012FA00D2AF120609C3E55C94FF40E90218367FB3
:10130A0002D27F11A2120609C2AFC27F11A2AE5C3D
:10131A00C3E55C947FD2AF500261AE1205F5C2AF4D
:10132A00120633D2AFDFDA11D9C3EE7897F6120676
:10133A000E1217B97F0AD27F11A2120609C2AFC2D2
:10134A007F11A2AE5CC3E55C947FD2AF50E6120572
:10135A00F5C2AF12061E1205FF12061ED2AFDFD665
:10136A0011D9EE24037896F6F87997E7C394824068
:10137A0003985006E824827897F612060E1216CCC5
:10138A001217E812060911A2C3E55C94FF50024144
:10139A00CB021836757C00757D00C3E55C954C4020
:1013AA0003855C4C12060978017988E7B403027850
:1013BA0005C3E55C98400241ABC2AF120633120680
:1013CA0033120633D2AF12060E753000E4F531F54A
:1013DA00320531E531F4703F0532789AE67819140E
:1013EA006012783214600D787D14600878FA1460FF
:1013FA0003753200C3E53298401D120F991205F5A4
:10140A00153275310078998673C2AF120633D2AF9E
:10141A00789886731206091205FFE52A700530745A
:10142A000221A278012074027806C3E55C9840A1E3
:10143A007888E6C394036003120609E52A7003025A
:10144A0011A2C2AF120F99E4F522F523F524F5256E
:10145A00F526F567D2AF7885E6C333F565E4F5443A
:0E146A00F545F546F547F548F570F52CF52DDE
:10147800F53775700875BB101205F512090730EDC0
:10148800FDA8BDA9BEE97001F8887112090B757035
:101498000875BB10111AC2AF7561FF1209A1852228
:1014A80061852262852263D2AF7522017524017598
:1014B8002501752601856069756A0175B69075A95B
:1014C80003757A017888E6B40307C27D307602D2C4
:1014D8007DD268D269753300120EEE120F1F120901
:1014E800C11209C81209C11209C81209C1120C5641
:1014F800120714120D57120D9E1209C8120C45300E
:101508006E031207702066031208BD3066031208C6
:10151800ED120D57120DCD1209C8120C56306E037C
:101528001207A5120D57120E461209C8120C4530A3
:101538006E03120803120D57120E771209C8120C07
:1015480056306E03120861120D57120EEE1209C8BA
:10155800120907120C45120D57120F1F12090B1210
:1015680009C8306932856461856462856069756A15
:101578000179187A0CC3E53399400FC269D26A8A97
:101588003585646185646302159FC3E55C940140F9
:10159800030214F502162D306A25206C22E5351455
:1015A8007006C26AD26B81F5F535C3E55C940140DB
:1015B800030214F57888E6C39403600302162D75B8
:1015C800360078FA79A4E760027803C3E55F98509B
:1015D80054307404E52A604D7888E6B40317207DFA
:1015E80005207607A1FD307602A1FD206C07D26C9C
:1015F800856461A13478F0306C058564617820C316
:10160800E54198500281F5306C1BC26CC27D307682
:1016180002D27DD26A75351285646181F50536E599
:101628005C6002C130753600C2AF120F997887E648
:10163800FE7602111A7887EEF6E4F522F523F524F2
:10164800F525F526F565752C00752D0075A900752D
:10165800B680757A00D2AF120609120F9978A4E6FF
:101668006006C292C291C290307409C3E5369404F0
:10167800400221A261D6901A0D782012170EE5209B
:10168800B4550CA312170EE520B4AA030216AC75C4
:101698007CA5757DF1120FAE1216CC757C00757D98
:1016A800000216CB901A0378807B0A12170EA30843
:1016B800DBF9901A0F788C7B1912170EA308DBF947
:1016C800901A2822C2AF12175112172E901A0074BE
:1016D8000E121713A37409121713A37415121713F4
:1016E800901A0378807B0A121712A308DBF9901A64
:1016F8000F788C7B19121712A308DBF912176412E2
:101708001742901A2822E493F622E6438F01538F5A
:10171800FDFFC3E583941C400122EF857CB7857DDE
:10172800B7F0538FFE22438F02438F01857CB78524
:101738007DB7901A0DF0538FFC22901A0D7455F155
:1017480013901A0E74AAF113227A3079D078209067
:101758001A40F10EE520F709A3DAF7227A3079D09A
:10176800901A40E7F11309A3DAF922AB74A875BB04
:1017780001027980BB02027981BB03027982BB0432
:10178800027984BB05027986BB06027992BB0702FF
:101798007987BB080279A3BB0902799CBB0A027945
:1017A80088BB0B027989E8F7227C0512060EDCFB60
:1017B80022C2AF12061E12062512062C120633127A
:1017C80005FF12061E12062512062C1206331205F4
:1017D800FF12061E12062512062C120633D2AF225D
:1017E800C2AF12063312062C12062512061E120567
:1017F800FF12063312062C12062512061E1205FFCA
:1018080012063312062C12062512061ED2AF22AE7D
:1018180074AF75C2AF12061E12061E12061E1205FE
:10182800FFDEF21206331205FFDFF8D2AF221217DD
:10183800B91217B11217B175740175750175760073
:1018480011177C05AD5C12060EC3ED955C70F5C3EF
:10185800E55C9401400AC3E55C94FF4037021879BF
:0E1868001217731216CC1217B9C2AF75EF1615
:101876001217B1DCD10576C3E5769403500280C217
:101886001217B10575E5741490009F93F808C3E527
:101896007598500280A91217B11217B10574C3E5E5
:1018A60074940C50028095120FAE1216CCC2AF750E
:0518B600EF161217B14E
:0319FD00021107CD
:101A00000E0915090904FF03FF0A03010155AA0184
:101A1000FFFFFFFFFF03FFFFFF25D0285004FF0259
:091A2000007AFF0101000300FF40
:101A4000234F76736B794D5232304150726F2320A1
:101A500023424C48454C492346333930232020202B
:101A60002020202020202020202020202020202076
:101C0000C2AFC2D353D9BF7581C043B20343FF8073
:101C1000752438752503B1DC7529A5752AF175E29F
:101C20004043F18053A47F75D4FFD2877DFA7803B7
:101C300079E67C10752200752300901DE97B0675FE
:101C400024987525013087028145208708D8FBD963
:101C5000F9DCF781B7308708D8FBD9F9DCF781B711
:101C6000B19CE493A3C39A6004DDC381B7DBDBB10D
:101C70008E6002812E7B08E493FAA3B16FDBF87AC1
:101C800030B16F752200752300B18EEAFCEBFDC305
:101C9000ED94FE400EB18E8A278B28ED30E0048A49
:101CA000828B83B18E7AC270D8C3ED94FE601950D6
:101CB000CEBD002BEC600F7520007521FF7529004B
:101CC000752A000200008100A827A9280809D80465
:101CD000D90281DCB192EA89AAF281CE0D81A3C337
:101CE000ED94035053EDA2E092007AC5C3E58294CF
:101CF00000E583941C508A200010438F02438F011B
:101D00008529B7852AB7F0300029A827A92808090E
:101D1000438F01538FFDD804D902A133C3E58394C7
:101D20001C4003A3A11689AAE28529B7852AB7F02A
:101D3000A3A116538FFC817F7AC1BD030CE493A34A
:101D4000FAB153DCF8B14B817F8181AA22AB23B178
:101D50006FEBFAEA6222752608C3E52313F523E543
:101D60002213F52250066323A0632201D526EAB18F
:101D7000DCB1DC75260AEAF4200102D287300102C8
:101D8000C287B1DCC3134002C201D526EB22B19257
:101D9000EAFB208702A192308702A197752608AE40
:101DA00024AF25C3EF13FFEE13FEB1E0B1DCC3EAAD
:101DB000133087024480FA30E703632201C3E5232E
:101DC00013F523E52213F52250066323A0632201B5
:101DD000D526D9E52265236523F52222AE24AF2539
:101DE0000E0FDEFEDFFCD20122424C48656C6934E6
:071DF000373164F390060196
:00000001FF
